:02000000A02935
:080008000B119C0003089D0090
:100010001D0883001C0809009400FF3A03193B28BF
:100020001408003A031D1B285C21950095039513C5
:10003000150888213B281408013A031D26285C2155
:100040009500950A9513150888213B281408803AD5
:10005000031D31285F2195009503951315088C2108
:100060003B281408813A031D3B285F219500950A1F
:10007000951315088C2108009400FF3A031977287E
:100080001408003A031D4E2862219500950395132C
:100090001508902162217F39AC2077281408013A95
:1000A000031D5C2862219500950A9513150890217F
:1000B00062217F39AC2077281408803A031D6A2812
:1000C00065219500950395131508942165218038C5
:1000D000AC2077281408813A031D77286521950004
:1000E000950A95131508942165218038AC200800E5
:1000F0009400941B872856210F3990389F005C216B
:1001000014077F39A00068217F39A1009228592166
:100110000F3990389F005F2114077F39A0006B21B1
:100120007F39A100D82008009400941BA1285621F3
:100130000F3990389F005C2114077F39A000A1017E
:10014000AA2859210F3990389F005F2114077F3961
:10015000A000A101D82008009400941BB9285621C2
:100160000F39C0389F0014087F39A0007F30A100EC
:10017000C22859210F39C0389F0014087F39A000C8
:100180007F30A100D82008009400941BCF2856216E
:100190000F39B0389F007B30A000A101D62859212B
:1001A0000F39C0389F007B39A000A101D82008007A
:1001B000FF30A2000310A10DA20D0314A10DA20D8A
:1001C0000310A00DA10DA20D0314A00DA10DA20DF1
:1001D00003109F0DA00DA10DA20D1E30950004303F
:1001E00000210314A20CA10CA00C9F0C031CFB28E3
:1001F00000008515FD288511FD28950BEF280800C6
:100200009400940B0129080019089B009B0C9B0C7F
:100210009B0C07309B051B08083885000301002153
:10022000060894001B080C3E84000008950019087D
:1002300044211405031D3129190844211505031D06
:10024000242900309A0043291908442196001609F0
:1002500095051B080C3E84001508800001309A00AB
:100260004329190844211505031D41291908442172
:1002700095041B080C3E84001508800002309A008B
:10028000432900309A00080007399700970A960121
:100290000314960D9703031D4929160808008312BD
:1002A00089008316081483120808080000304F21C3
:1002B000080001304F21080002304F2108000330B0
:1002C0004F21080004304F21080005304F2108005D
:1002D00006304F21080007304F2108000800831224
:1002E00089001808880083160812081555308900FF
:1002F000AA3089008814081E7B290811831208007F
:10030000980000306E210800980001306E2108002E
:10031000980002306E210800980003306E2108001A
:10032000980004306E210800980005306E21080006
:10033000980006306E210800980007306E210800F2
:10034000831285018601831600308500FF30860008
:100350005330810083129401950196019701980111
:1003600099019A019E019B01FF308C008D008E0047
:100370008F0090009100920093009F00A000A100C8
:10038000A2000030C4208030C420990104211A0842
:10039000003A0319262A1A08023A0319172A1908DB
:1003A0002F3C031CDF291908173C031CDB29190803
:1003B0007F397820262A190880387820262A1908BB
:1003C000303A031DE62900300C20162A1908313A6C
:1003D000031DED2901300C20162A1908323A031D9D
:1003E000F42980300C20162A1908333A031DFB2902
:1003F00081300C20162A1908343A031D022A0030D5
:100400003C20162A1908353A031D092A01303C20E0
:10041000162A1908363A031D102A80303C20162A65
:100420001908373A031D162A81303C20262A19085C
:100430002F3C031C262A1908173C031C232A1908E1
:100440007F399420262A190880389420990A403050
:080450001906031DC629C52988
:0840000005000900060007009D
:02400E00FA3F77
:104200000000000029002900000000007F007F005E
:104220004D004B004300200076002E0031002E0090
:10423000310020004A0044005000200028006300A4
:084240002900200032006B0090
:00000001FF
